:1000000019C033C032C031C030C030C03BC02DC079
:100010002CC02BC02AC048C328C027C026C025C07A
:1000200024C07DC4D2C289C2BAC21FC01EC01DC0B6
:100030001CC01BC011241FBECFEFD2E0DEBFCDBF5E
:1000400011E0A0E0B1E0E0E4FCE002C005900D9218
:10005000A630B107D9F712E0A6E0B1E001C01D92C9
:10006000AA32B107E1F718D0EAC5CACF1F920F92A2
:100070000FB60F921124109213010F900FBE0F9024
:100080001F9018951F920F920FB60F9211240F9088
:100090000FBE0F901F901895CDEFD2E0DEBFCDBF01
:1000A0001A82198205C089819A8101969A8389836F
:1000B00089819A818F5F9F4FB1F74E9901C025C703
:1000C0005AD0A0D06ED020D488E18093600087E021
:1000D00080936000789480910001882319F0109239
:1000E0000001D4D080911301882399F1F89412D49F
:1000F00042D01BD2BAD1909164008FEE80936400FD
:1001000080E480936D0084E08BBB80916800846004
:1001100080936800A89580EC8093600083B7817F0E
:10012000846083BF83B7816083BF7894889583B7E9
:100130008E7F83BFF89410926D0080E880936000FA
:1001400090936400E1D31092390181E08093000123
:1001500078948091390181112ED18091D201882328
:1001600009F4B9CF80911801A1E0B0E0082E5BD569
:100170001092D201B0CF15B883E184B918B88FE0DE
:1001800087B91BB886EA8AB985E08093C40080E409
:100190008093C0001092C1001092C20010926F00B4
:1001A00008959AE59093D6018091D6018093D50168
:1001B0008091D5018093D4019093D9018091D90188
:1001C0008093D8018091D8018093D70180EF8093EC
:1001D000DB018091DB018093DA011092160110920D
:1001E000170181E08093DD01A1E0B0E014D5802DFE
:1001F000992780931801209186012093DC01809338
:10020000DE010895A0E0B0E006D5802D9927809307
:100210001501883018F084E080931501089520E0DE
:1002200009C090E000000000000000009F5F9031D6
:10023000C9F72F5F2817A9F7089590E0E0EEF1E0E5
:100240008191980F82E0E832F807D1F79195909369
:10025000280208951F9358D15D9A80E000008F5FB7
:100260008F3FE1F720E010E006C0822F99278770CA
:100270009070892B19F4110F489911602F5F213468
:10028000A0F353D1812F99271F9108951F9380E0E8
:1002900090E0ACE2B1E0E9E1F1E08D9311920196DA
:1002A0008D309105D1F741D18AEFB9DF10E4109379
:1002B000C0001092C1001092C20026D184E0AFDFCE
:1002C0008091D101992701966DE070E07DD4FC0109
:1002D0008093D101FF27E45DFE4F808180938601EA
:1002E00080918601809316018091860160E0D4D0D0
:1002F000549885E294DF5D9A85E091DF1092D301F6
:100300001093C00080E98093C10086E48093C2000E
:1003100010E0B0D01092D00141D38091D0018F3F36
:10032000B1F58091D301882391F51092D00180918D
:100330001301882381F0E0910101F0910201818194
:1003400085FD03C092D0F1D034C0569A4E99FECFAD
:10035000109213015698209184003091850080916D
:10036000270190912801281B390B83E0220F331FAE
:100370008A95E1F782E794E0821B930B90938900C2
:100380008093880063D08FEF8093390112C08091F1
:10039000840090918500805A974108F4BECF8AD39B
:1003A00080911301882329F41F5F123009F0B1CF27
:1003B0007DCF1F9108954091290130913B012091FB
:1003C0003A01E9E1F1E0ACE2B1E05CE98081853637
:1003D00074F09C91F894935F01C099559935E8F7B2
:1003E0007894941710F03917A8F79C935083222320
:1003F00089F48C91841728F0381718F08081865F73
:1004000008C08081181614F4815003C0882311F0AD
:100410008F5F80833196119681E0E632F807B1F65E
:10042000222319F481E080933A0108958091D1014B
:10043000992701966DE070E0C7D38093D101ECE27B
:10044000F1E0E80FF11D8081992708951092850051
:10045000109284001092800082E08093810086BB1D
:1004600080936F0010920801089510926F0082E04F
:1004700086BB08951092850010928400109280002F
:100480001092820082E086BB10926F0083E080931E
:100490008100109208010895382F299A59985C9884
:1004A000419860FF07C080911501880F8167232F55
:1004B000255E11C020E090EA5C9897FF02C0599A2F
:1004C00001C059985C9A2F5F293011F0990FF4CF31
:1004D000232F245E84E35C989927982F882720682F
:1004E000820F911D20E05C9897FF02C0599A01C0CD
:1004F00059985C9A2F5F203119F0880F991FF3CF1C
:100500005C985998419A0895299A5A9A419A5D9807
:1005100028985C985998549A0895299A419A5D9818
:1005200028985C985998549A08955D982898299825
:100530005A9841985C98599808951F920F920FB657
:100540000F9211242F938F939F93EF93FF932091FA
:100550002902273011F429980CC0243551F48091D8
:1005600028029FE089278093C60088E48093C10019
:1005700009C0E22FFF27EC52FE4F80819FE08927C0
:100580008093C6002F5F20932902FF91EF919F91E6
:100590008F912F910F900FBE0F901F9018951F9263
:1005A0000F920FB60F9211248F9380E48093C000B6
:1005B0001092C1001092C20028984198299A8F91F8
:1005C0000F900FBE0F901F9018951F920F920FB6AD
:1005D0000F9211242F933F938F939F93EF93FF9349
:1005E0002091D0013091C6008FE038272430E9F403
:1005F00080910601E0910101F0910201E80FF11DE7
:1006000030838F5F809306019091D301930F909375
:10061000D3018934E1F580E48093C0001092C100D9
:100620001092C2005D982FEF32C02330C1F41092B7
:100630000601809184009091850090932801809319
:1006400027018091270190912801875A9B4F909311
:100650008900809388003093070124E018C0E22FBE
:10066000FF27EA5EFE4F8081381729F42F5F82E072
:10067000809312010CC0223039F43F3F29F481E00D
:100680008093120123E003C01092120120E0209316
:10069000D001FF91EF919F918F913F912F910F90FA
:1006A0000FBE0F901F9018951F920F920FB60F92CA
:1006B00011242F933F934F935F936F937F938F9367
:1006C0009F93AF93BF93EF93FF93809108018F5F48
:1006D000809308018150823009F4BDC0833030F42A
:1006E000882359F0813009F0F8C09AC0833009F4AA
:1006F000D3C0843009F0F1C0DBC080E48093C00037
:100700001092C1001092C20008DF80913A018F5F01
:1007100080933A019091D0019F3FB9F58091D30128
:10072000882399F55F9A9093390181E080932B019A
:10073000409107018091D101992701966DE070E009
:1007400043D2282F3327D901A45DBE4F8C9148177F
:1007500051F0493540F4F901E75EFE4F808187FD95
:1007600002C04C93108220910101309102018091CE
:100770000301909104019093020180930101309351
:10078000040120930301A7D11FC010922B01809177
:1007900039018823C9F08091390181508093390152
:1007A00080913901882341F45F9881E080930001B2
:1007B00010926F0082E086BBE091D101FF27E75ED7
:1007C000FE4F80818F5F8083809186012FDE809332
:1007D0008601809186018093DC018091D101992767
:1007E00001966DE070E0F0D1FC01E45DFE4F808188
:1007F0008093DF018091860161E04EDE80E480938A
:10080000C00088E08093C1008091880090918900A9
:1008100084589E4F90938900809388004BD15DC08F
:1008200080918800909189008C5B9A4F9093890009
:10083000809388001092290286E48093C200289A4F
:1008400088E28093C10085E58093C6008093C6004E
:100850007894F3DC42C061DEA1D080918601E6DDB0
:100860008093860180918601809316011092D001B9
:10087000109212011092D3018091860160E00CDE8B
:1008800080918800909189008B5D9E4F90938900A4
:1008900080938800549821C08091880090918900AD
:1008A000895A9F4F90938900809388005D9A15C064
:1008B0001092D30180E48093C00080E98093C1004E
:1008C00086E48093C20080918800909189008C5BBF
:1008D0009A4F90938900809388008091080165E089
:1008E00067D190930801FF91EF91BF91AF919F91D4
:1008F0008F917F916F915F914F913F912F910F90C9
:100900000FBE0F901F90189580EC8CBD5F98429899
:10091000409808951CBC5F984298409808951F9293
:100920000F920FB60F9211248F939F93EF93FF9323
:1009300080910F01E82FFF27E052FE4F9EB5908374
:10094000409A8F5F80930F01909110019F5F909369
:1009500010019150863071F48091E00180FF03C056
:1009600087E280930F0180911101882319F49E5D25
:100970009093100180911001E0910D01F0910E0112
:10098000E80FF11D80818EBD4098FF91EF919F91FE
:100990008F910F900FBE0F901F901895CF93DF93FC
:1009A00010920F0110921001A0910301B091040167
:1009B000B0930E01A0930D0180913901882379F441
:1009C000ED0129819091E1019695822F82958F709A
:1009D000892780FF42C080E1282729833EC080917B
:1009E0002B01882341F0FD018181887080930C01E7
:1009F00010920B010FC080910B01882341F01092DF
:100A00000C01FD013196ED012981247010C081E0B7
:100A100080930B01FD013196ED019981292F2470FE
:100A200080910C01882319F09460998303C0808120
:100A30008B7F808320930C0180912B01882329F0E8
:100A40008C9181708093110108C090E08091110118
:100A5000882309F491E0909311018C918EBD429A04
:100A6000DF91CF9108958091E101E0910301F09130
:100A700004019181869592959F70982790FF19C0E7
:100A80008091E201863B19F0873B99F405C0809183
:100A900018018093E30108958091E301882349F0D0
:100AA0008091E401882329F41092E20181E080938F
:100AB00013010895429880910A01882329F08091BA
:100AC000E10188608093E1018091E101847080936D
:100AD0000A01C9DF0895CF93DF938091120181301D
:100AE00059F48FEF8093DE0186EB8093E2018091D1
:100AF00018018093E30106C0823021F4809118012F
:100B00008093DE01E0910301F091040191818091D5
:100B1000E101969582958F70892780FF46C0DF019D
:100B200012968281883831F0853BE1F0843009F0FB
:100B30003CC026C08381ED019A819817B0F19935A8
:100B400010F088E58A83ED018A8123819927821B31
:100B50009109853591054CF5209329018A8180936F
:100B60003B0123C04E9921C083818093180181E00D
:100B70008093D20186EB82838FEF8093DE0115C0D4
:100B800090910901E92FFF27E051F14F20E0849176
:100B90008D932F5F31962430D1F7892F99270496B2
:100BA0006CE070E011D080930901DF91CF9108953E
:100BB000991B79E004C0991F961708F0961B881FAF
:100BC0007A95C9F78095089597FB092E07260AD0D4
:100BD00077FD04D00CD006D000201AF470956195F2
:100BE0007F4F0895F6F7909581959F4F0895AA1B22
:100BF000BB1B51E107C0AA1FBB1FA617B70710F008
:100C0000A61BB70B881F991F5A95A9F78095909539
:100C1000BC01CD010895F999FECFB2BDA1BDF89AEE
:100C2000119600B40895F999FECFB2BDA1BD00BCE4
:100C300011960FB6F894FA9AF99A0FBE0895FFCF5D
:060C4000013C01870100E8
:0C0EF000C8020900C9710904CA00000012
:00000001FF
